:100000000C9434000C9400000C9400000C9400003C
:100010000C9400000C9400000C9400000C94000060
:100020000C9400000C9400000C9400000C94000050
:100030000C9400000C94F3000C9400000C9400004D
:100040000C9400000C9400000C94C3000C94CD00A0
:100050000C94D9000C9400000C9400000C94000047
:100060000C9400000C9400000FEF0DBF08E00EBFD1
:1000700099278FEF0E94B1000FE107B998B97894E2
:1000800002C0FFCFF894A0E0B1E01091C100106968
:100090001093C100A330F1F71091C1001F761093A7
:1000A000C1009093C600409A0E94730060FDEBCFA0
:1000B00061FDE9CF62FD0E94880063FDE4CF64FD2D
:1000C000E2CF449AA0E0B1E01091C1001062109319
:1000D000C100A430F1F71091C10017791093C1004D
:1000E0009093C600D0CF009100010F7061E0002313
:1000F00019F0660F0A95FBCF7727009101010F7069
:10010000702B009102010F700295702B419A089597
:10011000429A709300017093010170930201A0E074
:10012000B1E01091C10010621093C100A430F1F74A
:100130001091C10017791093C1009093C600A0E000
:10014000B2E01091C10010691093C100A717F1F738
:100150001091C1001F761093C1009093C600439A7E
:1001600008959093C6009093C0009093C10090931F
:10017000C20010E01093C50013E31093C40016E012
:100180001093C20008951F935091C600152F107F41
:10019000103909F45D931F9118951F935D91509349
:1001A000C6001091C1001F7D18641093C1001F91FB
:1001B00018951F931091C100177B10621093C10016
:1001C0001F911895909380009093810090938200E6
:1001D000909385009093840090936F00909310010A
:1001E0009093110108953F93309110013395209120
:1001F0001201321719F43327809311013093100143
:040200003F9118957D
:00000001FF
